:100000004F07480720074C074F074F074B072107AB
:10001000200749077407270773072007720765073A
:1000200061076C0720076F0775077407700775076E
:1000300074072007660772076F076D0720074607DA
:100040005007470741072D07760774073107300728
:10005000300721072007200720072007DA07C407F9
:10006000C407C407BF072007DA07C407C407C407CB
:10007000C407C407C407C407C407C407C407C40728
:10008000C407C407C407C407C407C407C407C40718
:10009000C407C407C407C407C407C407C407BF070D
:1000A000410742074307440745074607470720071C
:1000B0002007300731073207200720076107620752
:1000C000630764076507660767072007200720079F
:1000D00021074007230724072507200720072007BB
:1000E0007E072007600720072B072007200720072F
:1000F000200720072007200720072007B3075F07F6
:100100005F075F07B3072007B3074E076F07200796
:100110007407650773077407200766076F07720780
:10012000200746874C8741875387488720077907F0
:100130006507740720072007200720072007B3075B
:10014000480749074A074B074C074D074E0720074A
:10015000200733073407350720072007680769079A
:100160006A076B076C076D076E07200720072007DB
:100170005E0726072A0728072907200720072007E8
:100180003B0720073A0720073D07200720072007E5
:10019000200720072007200720072007B3072D0787
:1001A0002D072D07B3072007B307200720072007D7
:1001B0002007200720072007200720072007200707
:1001C00020072007200720072007200720072007F7
:1001D0002007200720072007200720072007B30754
:1001E0004F07500751075207530754075507200779
:1001F0002007360737073807200720076F077007E3
:100200007107720773077407750720072007200717
:100210007B077D075B075D073C073E07200720073C
:10022000270720072207200720072007200720078D
:10023000200720072007200720072007B3075807BB
:1002400058075807B3072007B307200720072007E0
:100250002007200720072007200720072007200766
:100260002007200720072007200720072007200756
:100270002007200720072007200720072007B307B3
:10028000200756075707580759075A07200720071E
:1002900020072007300720072007200720077607C0
:1002A0007707780779077A072007200720072007B4
:1002B0002E072C072F073F075C077C072007200726
:1002C0002D0720075F0720072007200720072007AA
:1002D000200720072007200720072007B3077C07F7
:1002E0007C077C07B3072007B307200720072007F8
:1002F00020072007200720072007200720072007C6
:1003000020072007200720072007200720072007B5
:100310002007200720072007200720072007B30712
:1003200041076E076407200773076F076D076507AE
:10033000200763076F076C076F077507720773075E
:100340003A0720072007200720072007200720075B
:100350002007200720072007200720072007200765
:100360002007200720072007200720072007200755
:10037000200720072007200720072007C007C40701
:10038000C407C407D9072007C007C407C407C407A8
:10039000C407C407C407C407C407C407C407C40705
:1003A000C407C407C407C407C407C407C407C407F5
:1003B000C407C407C407C407C407C407C407D907D0
:1003C000DA02C402C402C402C402BF022007D60378
:1003D000C403C403C403B70320072007D604B7042B
:1003E0002007D605B7052007D606B706D607B707F4
:1003F000D608B708D609B709D60AB70AD60BB70B7D
:10040000D60CB70CD60DB70DD60EB70ED60FB70F4C
:1004100020072007200720072007200720072007A4
:100420002007200720072007200720072007200794
:100430002007200720072007200720072007200784
:100440002007200720072007200720072007200774
:100450002007200720072007200720072007200764
:10046000B3022007200720072007B3022007BA03A2
:10047000200720072007BA0320072007D304BD0464
:100480002007D305BD052007D306BD06D307BD074A
:10049000D308BD08D309BD09D30ABD0AD30BBD0BD0
:1004A000D30CBD0CD30DBD0DD30EBD0ED30FBD0FA0
:1004B0002007200720072007460747072007630774
:1004C0006F076C076F077507720773072007200710
:1004D00020072007200720072007200720072007E4
:1004E00020072007200720072007200720072007D4
:1004F00020072007200720072007200720072007C4
:10050000C002C402C402C402C402D9022007D30339
:10051000C403C403C403BD0320072007200720072A
:100520002007200720072007200720072007200793
:100530002007200720072007200720072007200783
:100540002007200720072007200720072007200773
:100550002007200720072007200720072007200763
:100560002007200720072007200720072007200753
:100570002007200720072007200720072007200743
:100580002007200720072007200720072007200733
:100590002007200720072007200720072007200723
:1005A0002007200720072007200720072007200713
:1005B0002007200720072007200720072007200703
:1005C00020072007200720072007200720072007F3
:1005D00020072007200720072007200720072007E3
:1005E00020072007200720072007200720072007D3
:1005F00020072007200720072007200720072007C3
:1006000020072007200720072007200720072007B2
:1006100020072007200720072007200720072007A2
:100620002007200720072007200720072007200792
:100630002007200720072007200720072007200782
:10064000D61FB71FD62FB72FD63FB73FD64FB74FBE
:10065000D65FB75FD66FB76FD67FB77FD60FB70FAE
:100660002007200742074707200763076F076C072B
:100670006F07750772077307200720072007C91443
:10068000BB142007C91EBB1E2007C92EBB2E200786
:10069000C925BB252007C91BBB1B2007C95FBB5F42
:1006A0002007C94FBB4F2007740F6F0F670F650FEF
:1006B000740F680F650F720F200F610F740F200FFA
:1006C0006C0F610F730F740F210F20072007200795
:1006D00020072007200720072007200720072007E2
:1006E000D31FBD1FD32FBD2FD33FBD3FD34FBD4F12
:1006F000D35FBD5FD36FBD6FD37FBD7FD30FBD0F02
:1007000020072007200720072007200720072007B1
:100710002007200720072007200720072007C814EC
:10072000BC142007C81EBC1E2007C82EBC2E2007E4
:10073000C825BC252007C81BBC1B2007C85FBC5FA1
:100740002007C84FBC4F200720072007200720079D
:100750002007200720072007200720072007200761
:100760002007200720072007200720072007200751
:100770002007200720072007200720072007200741
:100780002007200720072007200720072007200731
:100790002007200720072007200720072007200721
:1007A0002007200720072007200720072007200711
:1007B0002007200720072007200720072007200701
:1007C00020072007200720072007200720072007F1
:1007D00020072007200720072007200720072007E1
:1007E00020072007200720072007200720072007D1
:1007F0002007200720072007C50F2007CE0F20075E
:10080000D80F2007D70F2007E80F2007E90F200790
:100810009B0F20079C0F2007990F2007EF0F200741
:100820002007200720072007200720072007200790
:100830002007200720072007200720072007200780
:100840002007200720072007200720072007200770
:100850002007200720072007200720072007200760
:100860002007200720072007200720072007200750
:100870002007200720072007200720072007200740
:100880002007200720072007200720072007200730
:100890002007200720072007200720072007200720
:1008A0002007200720072007200720072007200710
:1008B0002007200720072007200720072007200700
:1008C00054076F076F0720076D07750763076807F1
:1008D00020076F07660720076107200767076F0774
:1008E0006F07640720077407680769076E076707C3
:1008F000200769077307200757074F074E0744076C
:1009000045075207460755074C07210720072D07C3
:1009100020074D076107650720075707650773071D
:10092000740720072007200720072007200720073B
:100930002007200720072007D60F2007B70F200722
:10094000D30F2007BD0F2007C40F2007BA0F2007C1
:10095000C70F2007B60F2007D00F2007D20F2007A0
:10096000200720072007200720072007200720074F
:10097000200720072007200720072007200720073F
:10098000200720072007200720072007200720072F
:10099000200720072007200720072007200720071F
:1009A000200720072007200720072007200720070F
:1009B00020072007200720072007200720072007FF
:1009C00020072007200720072007200720072007EF
:1009D0002007200720072007200F200F200F200FBF
:1009E000200F200F200F200F200F200F200F200F8F
:1009F000200F200F200F200F200F200F200F200787
:100A0000B00FB00FB00FB10FB10FB10FB20FB20FE7
:100A1000B20FDB0FDB0FDB0FDF0FDF0FDF0FDC0FA2
:100A2000DC0FDC0FDD0FDD0FDD0FDE0FDE0FDE0F65
:100A3000200720072007200720072007200720077E
:100A4000200720072007200720072007200720076E
:100A5000200720072007200720072007200720075E
:100A6000200720072007200720072007200720074E
:100A70002007200720072007D50F2007B80F2007E1
:100A8000D40F2007BE0F2007CD0F2007B30F20077C
:100A9000C60F2007B50F2007CF0F2007D10F200763
:100AA000200720072007200720072007200720070E
:100AB00020072007200720072007200720072007FE
:100AC00020072007200720072007200720072007EE
:100AD00020072007200720072007200720072007DE
:100AE00020072007200720072007200720072007CE
:100AF00020072007200720072007200720072007BE
:100B000020072007200720072007200720072007AD
:100B1000200720072007200720072007200720079D
:100B2000200720072007200720072007200720078D
:100B3000200720072007200720072007200720077D
:100B4000010F2007020F2007030F2007040F2007C3
:100B5000050F2007060F2007F00F20077F0F200743
:100B60000E0F20070F0F2007E30F2007F10F2007BC
:100B7000F40F2007F50F2007EA0F20079D0F20072D
:100B8000E40F2007F80F2007FB0F2007FC0F2007BA
:100B9000830F2007840F2007850F2007A00F200751
:100BA000A60F2007860F20078E0F20078F0F200724
:100BB000910F2007920F2007C50F2007CE0F2007A7
:100BC000D80F2007D70F2007E80F2007E90F2007CD
:100BD0009B0F20079C0F2007990F2007EF0F20077E
:100BE00020072007200720072007200720072007CD
:100BF00020072007200720072007200720072007BD
:100C000020072007200720072007200720072007AC
:100C1000200720072007200720072007200720079C
:100C2000200720072007200720072007200720078C
:100C3000200720072007200720072007200720077C
:100C4000200720072007200720072007200720076C
:100C5000200720072007200720072007200720075C
:100C6000200720072007200720072007200720074C
:100C7000200720072007200720072007200720073C
:100C8000180F2007190F20071E0F20071F0F20071E
:100C9000100F2007110F2007120F20071D0F20072C
:100CA000140F2007150F2007E00F2007E10F200782
:100CB000E20F2007E50F2007E60F2007E70F2007C8
:100CC000EB0F2007EC0F2007ED0F2007EE0F20079A
:100CD000880F2007890F20078A0F2007820F20071F
:100CE000900F20078C0F20078B0F20078D0F2007F8
:100CF000A10F20079E0F2007DA0F2007BF0F200744
:100D0000C00F2007D90F2007C40F2007B30F2007FB
:100D1000C30F2007B40F2007C10F2007C20F200701
:100D2000200720072007200720072007200720078B
:100D3000200720072007200720072007200720077B
:100D4000200720072007200720072007200720076B
:100D5000200720072007200720072007200720075B
:100D6000200720072007200720072007200720074B
:100D7000200720072007200720072007200720073B
:100D8000200720072007200720072007200720072B
:100D9000200720072007200720072007200720071B
:100DA000200720072007200720072007200720070B
:100DB00020072007200720072007200720072007FB
:100DC000AE0F2007AF0F2007F20F2007F30F200709
:100DD000A90F2007AA0F2007FD0F2007F60F2007F5
:100DE000AB0F2007AC0F2007800F2007870F2007CD
:100DF000A50F2007A40F2007980F20079F0F20079B
:100E0000F70F2007F90F2007AD0F2007A80F2007C5
:100E1000930F2007940F2007950F2007A20F20079C
:100E2000A70F2007960F2007810F2007970F200795
:100E3000A30F20079A0F2007C90F2007BB0F200719
:100E4000C80F2007BC0F2007CD0F2007BA0F2007BF
:100E5000CC0F2007B90F2007CA0F2007CB0F2007A0
:100E6000200720072007200720072007200720074A
:100E7000200720072007200720072007200720073A
:100E8000200720072007200720072007200720072A
:100E9000200720072007200720072007200720071A
:100EA000200720072007200720072007200720070A
:100EB00020072007200720072007200720072007FA
:100EC00020072007200720072007200720072007EA
:100ED00020072007200720072007200720072007DA
:100EE00020072007200720072007200720072007CA
:100EF00020072007200720072007200720072007BA
:100F000042074F07540754074F074D0720074C0768
:100F100049074E074507200742074F075407540764
:100F20004F074D0720074C0749074E074507200785
:100F300042074F07540754074F074D0720074C0738
:100F400049074E074507200742074F075407540734
:100F50004F074D0720074C0749074E074507200755
:100F60002D072D072D072D072D072D072D072D07E1
:100F70002D072D072D072D072D072D072D072D07D1
:100F80002D072D072D072D072D072D072D072D07C1
:100F90002D072D072D072D072D072D073E072007AD
:100FA0000000000000000000000000000000000041
:100FB0000000000000000000000000000000000031
:100FC0000000000000000000000000000000000021
:100FD0000000000000000000000000000000000011
:100FE0000000000000000000000000000000000001
:100FF00000000000000000000000000000000000F1
:00000001FF
